:020000040800F2
:10000000E007002045170008FD020008FF02000875
:1000100003030008070300080B03000800000000AA
:100020000000000000000000000000000F030008B6
:100030001103000800000000130300081503000866
:100040005F1700085F1700085F1700085F170008B8
:100050005F1700085F1700085F1700085F170008A8
:100060005F1700085F1700085F1700085F17000898
:100070005F1700085F1700085F1700085F17000888
:100080005F1700085F1700085F1700085F17000878
:100090005F1700085F1700085F1700085F17000868
:1000A0005F1700085F1700085F1700085F17000858
:1000B0005F1700085F1700085F1700085F17000848
:1000C0005F1700085F1700085F1700085F17000838
:1000D0005F1700087F20000897200008D52000083F
:1000E0005F1700085F1700085F17000800F002F8AC
:1000F00000F03FF80AA090E8000C82448344AAF183
:100100000107DA4501D100F034F8AFF2090EBAE880
:100110000F0013F0010F18BFFB1A43F0010318473B
:10012000D4210000F4210000103A24BF78C878C11F
:10013000FAD8520724BF30C830C144BF04680C60ED
:10014000704700000023002400250026103A28BF35
:1001500078C1FBD8520728BF30C148BF0B60704739
:10016000732902F06480002070471FB51FBD10B5D1
:1001700010BD02F08FF81146FFF7F7FF00F04CF8C2
:1001800002F0ADF803B4FFF7F2FF03BC01F03AFE52
:1001900010B552A001F0BAFF4FF4967001F0FFFDC8
:1001A00050A1514802F01BF804464CA001F0AEFFEC
:1001B0004FF4967001F0F3FD4AA14B4802F00FF89E
:1001C000044601F015FBC4B90120484908604FF40A
:1001D000967001F0E4FD4FF4967001F0E0FD4FF4ED
:1001E000967001F0DCFD4FF4967001F0D8FD002010
:1001F0003F49C1F8800101F0FBFA38A001F086FF09
:100200004FF4967001F0CBFD01F0F2FA35A13648BB
:1002100001F0E5FF044610BD86B001F083FD01F05A
:10022000EBFD01F0AFFA4FF4E13001F015FE4FF4B1
:10023000E13001F060FE40F27121072001F0C6FAC2
:1002400000BF01F050FD0028FBD1FFF7A1FF01F036
:10025000E6FA01F0A1FB3FE004A905A801F017FDB3
:100260009DF814000A2190FBF1F03030C0B28DF8F7
:1002700004009DF8140090FBF1F201FB12003030F5
:10028000C0B28DF805009DF8100090FBF1F0303001
:10029000C0B28DF806009DF8100090FBF1F201FB52
:1002A00012003030C0B28DF8070000208DF8080031
:1002B00001A910A001F08FFB01F0CBFB4FF4FA7005
:1002C00001F06DFD0C48006808B9012000E0002035
:1002D0000949086001F08CFABEE7000041540D0A9C
:1002E000000000004F4B0000B700002080012142B9
:1002F000000021423400000080812142704700BF8D
:10030000FEE700BFFEE700BFFEE700BFFEE7704765
:10031000704770477047000010B500F03DFE0120A7
:1003200000F0BFFE00BF212000F079FE0028FAD0C7
:10033000102000F099F9022000F082F9002000F06E
:10034000D0FE002000F0DFFE4FF4806000F0D2FE0F
:100350004FF46011002000F0A7FE012000F0B0FE75
:1003600000BF392000F05BFE0028FAD0022000F028
:10037000AAFE00BF00F0B0FE0828FBD101211D201D
:1003800000F078FF10BD0CB50020019000906C4883
:10039000006840F480306A49086000BF684800681F
:1003A00000F4003000900198401C0190009818B9AA
:1003B0000198B0F5A06FF1D16148006800F40030F9
:1003C00010B10120009001E0002000900098012869
:1003D00043D15C48006840F010005A490860084664
:1003E000006820F0030008600846006840F0020042
:1003F0000860534840685249486008464068486071
:100400000846406840F4806048600846406820F430
:100410007C1048600846406840F4E8104860084690
:10042000006840F08070086000BF4548006800F038
:1004300000700028F9D04248406820F0030040498D
:1004400048600846406840F00200486000BF3C48F1
:10045000406800F00C000828F9D10CBD10B5FFF77A
:1004600092FF10BD10B53648006840F001003449D5
:1004700008600846406834490840314948600846E9
:100480000068324908402E4908600846006820F498
:10049000802008600846406820F4FE0048604FF461
:1004A0001F008860FFF7DAFF4FF0006028490860FE
:1004B00010BD10B5002100200022214B5B6803F025
:1004C0000C0121B1042906D0082928D107E0214BCD
:1004D000214C236027E01F4B1F4C236023E0184B67
:1004E0005B6803F47010164B5B6803F480320223E0
:1004F00003EB904022B9194B4343174C23600DE0A6
:100500000F4B5B6803F4003323B1144B4343124C8D
:10051000236003E00F4B43430F4C236003E00D4B7C
:100520000D4C236000BF00BF054B5B68C3F3031392
:100530000B4CE15C084B1B68CB40074C236010BDA3
:1005400000100240002002400000FFF8FFFFF6FE0E
:1005500008ED00E000127A000000002000093D00D4
:100560000400002031490143314A1160704770B5E1
:10057000002100230F22C47804B32D4C246804F416
:10058000E064C4F5E064210AC1F10403CA40447880
:1005900004FA03F18478144021430901254C0678BC
:1005A000A155047804F01F050124AC4005786D11B5
:1005B000AD0005F1E025C5F8004109E0047804F03C
:1005C0001F050124AC401C4D0678761145F82640E5
:1005D00070BD1A4A0A400243154B1B1F1A60704730
:1005E00039B1134A121D12680243114B1B1D1A60C8
:1005F00006E00F4A121D126882430D4B1B1D1A6044
:100600007047042808D14FF0E021096941F0040146
:100610004FF0E022116107E04FF0E021096921F07D
:1006200004014FF0E0221161704700000000FA055C
:100630000CED00E000E400E080E100E080FFFF1F3F
:1006400001460020FE4A106800F0380008431060A0
:100650007047FB49096821F00801F94A1160114609
:100660000968014311607047F549096821F01001DC
:10067000F34A116011460968014311607047F1485F
:10068000EF494860F04848607047EE48EC494860E0
:10069000ED4848607047EA48006940F08000E8494A
:1006A00008617047E648006940F08000E44908614D
:1006B00070470420E249C96801F0010109B1012035
:1006C0000EE0DF49C96801F0040109B1022007E02A
:1006D000DB49C96801F0100109B1032000E00420E2
:1006E000704700B502460423FFF7E3FF034603E02B
:1006F000FFF7DFFF0346521E012B01D1002AF7D17D
:1007000002B90523184600BD30B5044604254FF450
:100710003020FFF7E6FF0546042D17D1C8480069D1
:1007200040F00200C649086108464461006940F093
:10073000400008614FF43020FFF7D3FF0546C04862
:10074000006941F6FD710840BD490861284630BD89
:1007500010B504244FF43020FFF7C3FF0446042CE7
:1007600016D1B748006940F00400B5490861084651
:10077000006940F0400008614FF43020FFF7B1FFFE
:100780000446AF48006941F6FB710840AC49086176
:10079000204610BD00B502460423FFF78AFF03463A
:1007A00003E0FFF786FF0346521E012B01D1002A0A
:1007B000F7D102B90523184600BD10B504244FF443
:1007C0003020FFF7E7FF0446042C16D19C4800694F
:1007D00040F004009A4908610846006940F0400072
:1007E00008614FF43020FFF7D5FF044694480069B4
:1007F00041F6FB71084092490861204610BD002077
:100800008F49C96901F0020109B1012000E000200F
:10081000704730B5A5250424FFF7F1FF00B100258E
:100820004FF43020FFF75DFF0446042C3AD1854891
:1008300083498860844888600846006940F0200049
:1008400008610846006940F0400008614FF430201C
:10085000FFF747FF0446042C1BD17948006941F695
:10086000DF710840764908610846006940F01000D1
:10087000086176480580E002FFF733FF0446052C47
:1008800010D06F48006941F6EF7108406C4908616B
:1008900008E0052C06D06A48006941F6EF7108406F
:1008A00067490861204630BD78B506460C460425E8
:1008B00000200090E802FFF714FF0546042D24D124
:1008C0005F48006940F001005D4908613480E8023A
:1008D000FFF707FF0546042D10D1B01C0090200C37
:1008E00000990880E802FFF7FCFE054654480069BD
:1008F00041F6FE7108405249086106E0504800691F
:1009000041F6FE7108404E490861284678BD70B531
:1009100004460D460426F002FFF7E3FE0646042EC9
:1009200011D14748006940F0010045490861258020
:10093000F002FFF7D6FE06464148006941F6FE7117
:1009400008403F490861304670BD70B505460E4607
:100950000424E002FFF7C5FE0446042C17D13948F1
:1009600037498860384888600846006940F01000C0
:1009700008612E80E002FFF7B4FE0446052C06D085
:100980002F48006941F6EF7108402D490861204663
:1009900070BD2DE9F04304464FF6FF763746B0466A
:1009A000B1460425E443E6B2C4F30727C4F307487D
:1009B0004FEA1469E802FFF794FE0546042D49D179
:1009C00020481F498860204888600846006940F038
:1009D00010000861FF2E06D01C4808300680E8028F
:1009E000FFF77FFE0546042D08D1FF2F06D01748DC
:1009F0000A300780E802FFF774FE0546042D0AD18D
:100A0000B8F1FF0F07D011480C30A0F80080E802C1
:100A1000FFF767FE0546042D0AD1B9F1FF0F07D095
:100A20000A480E30A0F80090E802FFF75AFE05468B
:100A3000052D0FD00248006941F6EF71084007E02C
:100A40000020024023016745AB89EFCD00F8FF1F6E
:100A5000664908612846BDE8F08330B505460424A0
:100A60004FF43020FFF73DFE0446042C41D160488E
:100A70005E4988605F4888600846006940F0200051
:100A800008610846006940F0400008614FF43020DA
:100A9000FFF727FE0446042C22D15448006941F692
:100AA000DF710840514908610846006940F01000B4
:100AB00008611DB100205049088002E0A5204E4980
:100AC00008804FF43020FFF70CFE0446052C10D0B0
:100AD0004648006941F6EF7108404449086108E062
:100AE000052C06D04148006941F6DF7108403F49B6
:100AF0000861204630BDF0B505460E461746042471
:100B00003B483A4988603B488860E002FFF7E9FDCE
:100B10000446042C19D13548006940F010003349CF
:100B2000086147F0F800304328433349891C0880A6
:100B3000E002FFF7D6FD0446052C06D02B480069DD
:100B400041F6EF710840294908612046F0BD274869
:100B5000C069800870472548006A70470020234913
:100B6000096801F0200109B1012000E00020704770
:100B700029B11E4A126902431C4B1A6104E01B4A48
:100B800012698243194B1A617047014600200129FE
:100B900008D1164AD26902F001020AB1012008E028
:100BA000002006E0114AD2680A400AB1012000E0A4
:100BB000002070470D49C860704704200B49C96880
:100BC00001F0010109B101200EE00849C96801F0F6
:100BD000040109B1022007E00449C96801F01001CD
:100BE00009B1032000E0042070470000002002400B
:100BF00023016745AB89EFCD00F8FF1F10B5044610
:100C0000CC48844208D10121042000F04DFB002192
:100C1000042000F049FB46E0C748844208D1012186
:100C2000082000F041FB0021082000F03DFB3AE0E5
:100C3000C248844208D10121102000F035FB002178
:100C4000102000F031FB2EE0BD48844208D1012184
:100C5000202000F029FB0021202000F025FB22E0CD
:100C6000B848844208D10121402000F01DFB00213A
:100C7000402000F019FB16E0B348844208D101215E
:100C8000802000F011FB0021802000F00DFB0AE025
:100C9000AE48844207D10121801500F005FB0021F8
:100CA000A01500F001FB10BD10B50121084600F0B1
:100CB000FBFA0021012000F0F7FA10BD2DE9F04108
:100CC000024600250026002000230024002791F87A
:100CD00003C00CF00F0591F803C00CF0100CBCF130
:100CE000000F03D091F802C04CEA050591F800C04E
:100CF000BCF1000F31D0146800202BE04FF0010C44
:100D00000CFA00F3B1F800C00CEA03069E4220D1B1
:100D100083004FF00F0C0CFA03F7BC4305FA03FCF9
:100D20004CEA040491F803C0BCF1280F06D14FF03F
:100D3000010C0CFA00FCC2F814C00AE091F803C0E0
:100D4000BCF1480F05D14FF0010C0CFA00FCC2F8C1
:100D500010C0401C0828D1D31460B1F800C0BCF109
:100D6000FF0F34DD546800202EE000F1080C4FF036
:100D7000010808FA0CF3B1F800C00CEA03069E4221
:100D800021D183004FF00F0C0CFA03F7BC4305FA96
:100D900003FC4CEA040491F803C0BCF1280F05D110
:100DA00000F1080C08FA0CF8C2F8148091F803C09E
:100DB000BCF1480F07D100F1080C4FF0010808FA08
:100DC0000CF8C2F81080401C0828CED35460BDE84F
:100DD000F0814FF6FF710180022181700421C17002
:100DE00070470246002093680B400BB1012000E0E1
:100DF000002070470146886880B270470246002094
:100E0000D3680B400BB1012000E000207047014681
:100E1000C86880B2704701617047416170470AB18C
:100E2000016100E041617047C16070474FF480325A
:100E30000A438261816182618269826970470246E8
:100E40000020434B18684FF68073184040EA0210A8
:100E500008433F4B186070473E49C8617047F0B582
:100E60000A46002300240021002500F00046B6F1C8
:100E7000004F02D1364EF16901E0354E7168C0F382
:100E8000034583B200F44016B6F5401F08D121F0A7
:100E900070612F4E766826F070662D4F7E6012E0EE
:100EA00000F48016B6F5801F06D1032606FA05F475
:100EB000A14341F0706106E0460D360103FA06F6E3
:100EC000B14341F0706122B1460D360103FA06F6D6
:100ED000314300F00046B6F1004F02D11C4EF161E3
:100EE00001E01B4E7160F0BD30B500228B071C0F76
:100EF0000F2303FA04F2164B08338C1053F82430F6
:100F00009343134C08348D1044F8253023468C103D
:100F100053F824308C07240F00FA04F423430C4CBC
:100F200008348D1044F8253030BD0A49DC310860A2
:100F30007047000000080140000C01400010014013
:100F40000014014000180140001C01400020014035
:100F500000000140000020420E49086070470D4922
:100F6000486070470B49886070474AF6AA200949D3
:100F7000086070474CF6CC4006490860704701464F
:100F80000020044AD2680A400AB1012000E0002093
:100F90007047000000300040DF48006840F001006A
:100FA000DD49086008464068DC490840DA49486085
:100FB00008460068DA490840D749086008460068D2
:100FC00020F4802008600846406820F4FE00486055
:100FD0004FF41F0088607047CF49096821F48031C1
:100FE000CD4A11601146096821F480211160B0F5E5
:100FF000803F03D0B0F5802F0ED106E0C6490968C6
:1010000041F48031C44A116007E0C349096841F4E2
:10101000A021C14A116000E000BF00BF704710B5B9
:1010200001460022002300204A11012A02D1BA4CB5
:10103000236806E0022A02D1B74C236A01E0B64CCD
:10104000636A01F01F02012494401C400CB101208E
:1010500000E0002010BD38B50020009000240025DD
:1010600000BF3120FFF7DBFF05460098401C0090D1
:101070000098B0F5A06F01D0002DF2D03120FFF71D
:10108000CEFF08B1012400E00024204638BD01460F
:101090000020A14A106820F0F80040EAC10010606A
:1010A0007047A04908607047024600209A4B586874
:1010B00020F47C1042EA01031843974B58607047B4
:1010C00098490866704701460020934A506820F00E
:1010D00003000843506070478F48406800F00C00E0
:1010E0007047014600208C4A506820F0F000084309
:1010F0005060704701460020874A506820F4E06045
:1011000008435060704701460020834A506820F42D
:10111000605040EAC1005060704729B17E4A527A5F
:1011200002437D4B5A7204E07B4A527A82437A4BE7
:101130005A7270477B49D8310860704701460020D9
:10114000754A506820F440400843506070470021C1
:10115000714A20321170704A82F82010012802D0A2
:1011600004280AD104E001216B4A2032117005E005
:101170000521694A2032117000E000BF00BF7047AE
:101180006949086070476449096A0143624A11620B
:101190007047654944390860704730B50021002226
:1011A000002400235C4D6D6805F00C0121B1042979
:1011B00005D0082923D105E05C4D056022E05B4D98
:1011C00005601FE0544D6D6805F47012524D6D6856
:1011D00005F48034022505EB92421CB9544D554369
:1011E00005600BE04C4D6D6805F400351DB1504DA8
:1011F0005543056002E04D4D5543056002E04B4DFF
:10120000056000BF00BF444D6D6805F0F00109099D
:10121000484D6B5C0568DD4045603F4D6D6805F4E9
:10122000E061090A434D6B5C4568DD4085603A4DDD
:101230006D6805F46051C90A3E4D6B5C4568DD4040
:10124000C560354D6D6805F44041890B3A4D6B5CC6
:10125000C568B5FBF3F5056130BD29B12E4A526969
:1012600002432D4B5A6104E02B4A526982432A4BB8
:101270005A61704729B1284A92690243264B9A6104
:1012800004E0254A92698243234B9A61704729B151
:10129000214AD2690243204BDA6104E01E4AD26936
:1012A00082431D4BDA61704729B11B4AD268024361
:1012B000194BDA6004E0184AD2688243164BDA60B0
:1012C000704729B1144A12690243134B1A6104E0B2
:1012D000114A12698243104B1A6170471249403912
:1012E000086070470F49C86470470B49C871704760
:1012F0000948406A40F080700749486270470146DB
:101300000020054A92680A400AB1012000E000204E
:101310007047014988727047001002400000FFF8D2
:10132000FFFFF6FE000042428004424200127A00B3
:1013300000093D00140000202400002010B50446E0
:10134000FB48844209D101218803FFF7ADFF00214A
:101350004FF48040FFF7A8FF32E0F648844209D1FD
:1013600001214804FFF7ADFF00214FF40030FFF7E3
:10137000A8FF25E0F048844209D101218804FFF745
:10138000A0FF00214FF48020FFF79BFF18E0EB48FF
:10139000844209D10121C804FFF793FF00214FF4D3
:1013A0000020FFF78EFF0BE0E548844208D10121C1
:1013B0000805FFF786FF00214FF48010FFF781FF3B
:1013C00010BD2DE9F04786B005460E460024A24622
:1013D00000BFA1460027B08900B100BF2F462C8A6C
:1013E0004CF6FF700440F08804432C82AC894EF622
:1013F000F3100440B08831890843718908430443DD
:10140000AC81AC8A4FF6FF400440B0890443AC8203
:1014100001A8FFF7C2FEC648874202D1DDF810A03E
:1014200001E0DDF80CA0A88900F4004040B10AEB0F
:10143000CA0000EB0A1031684900B0FBF1F807E080
:101440000AEBCA0000EB0A1031688900B0FBF1F822
:101450006420B8FBF0F004012009642101FB10892D
:10146000A88900F4004040B1322000EBC900B0FB75
:10147000F1F000F00700044308E0322000EB09100F
:101480006421B0FBF1F000F00F0004432C8106B0A2
:10149000BDE8F0874FF41651016000218180C180C2
:1014A00001810C21418100218181704710B50246E4
:1014B0000020108A4FF2FF0318400B884C8823430A
:1014C0008C882343CC8823431843108210BD00210D
:1014D000018041808180C180704721B1828942F4BE
:1014E0000052828104E082894DF6FF731A408281A6
:1014F0007047F0B50346002400260025002040F682
:101500006A17B94200D100BF1846C1F3421401F076
:101510001F06012707FA06F5012C01D10C3004E063
:10152000022C01D1103000E014301AB107682F43AB
:10153000076002E00768AF430760F0BD1AB1838A15
:101540000B43838202E0838A8B4383827047028A43
:101550004FF6F0731A400282028A0A4302827047F1
:1015600082894FF2FF731A40828182890A43828105
:10157000704721B1828942F00202828104E08289AF
:101580004FF6FD731A4082817047028A4FF6DF736F
:101590001A400282028A0A430282704721B1028AFB
:1015A00042F48042028204E0028A4BF6FF731A4042
:1015B00002827047C1F30802828070470146888822
:1015C000C0F308007047818941F0010181817047B3
:1015D000028BD2B20283028B42EA0122028370475D
:1015E000028B02F47F420283028B0A43028370471C
:1015F00021B1828A42F02002828204E0828A4FF680
:10160000DF731A408282704721B1828A42F0100251
:10161000828204E0828A4FF6EF731A40828270471A
:1016200021B1828A42F00802828204E0828A4FF667
:10163000F7731A408282704721B1828942F40042D6
:10164000828103E08289C2F30E028281704721B158
:10165000828A42F40062828204E0828A4FF2FF733F
:101660001A4082827047828A4FF6FB731A40828248
:10167000828A0A438282704721B1828A42F0020242
:10168000828204E0828A4FF6FD731A40828270479C
:1016900002460020B1F5007F00D100BF13880B4047
:1016A0000BB1012000E00020704701F40072B2F598
:1016B000007F00D100BFCA430280704770B5024668
:1016C000002400230025002040F66A16B14200D114
:1016D00000BFC1F3421501F01F03012606FA03F310
:1016E000012D02D19689334006E0022D02D1168ADF
:1016F000334001E0968A33400C12012606FA04F4C6
:101700001688344013B10CB1012000E0002070BDF8
:1017100010B50022002340F66A14A14200D100BF98
:101720000A1201249440A3B2DC43048010BD0000DF
:10173000003801400044004000480040004C004098
:10174000005000400948804709480047FEE7FEE78F
:10175000FEE7FEE7FEE7FEE7FEE7FEE7FEE7FEE761
:1017600004480549054A064B704700006504000817
:10177000ED000008E0010020E0070020E003002069
:10178000E003002008B501210C20FFF773FD0120C4
:10179000ADF8000010208DF8030003208DF8020042
:1017A00069460848FFF78AFA0120ADF800001020CA
:1017B0008DF8030003208DF8020069460248FFF708
:1017C0007DFA08BD000C01400008014070B50546D7
:1017D0000C4645F25550FFF7BFFB2846FFF7BFFB0D
:1017E0002046FFF7BFFBFFF7C0FBFFF7C3FB70BD51
:1017F00010B5FFF7BAFB10BD10B59C4800F01DFCFA
:10180000002404E0002099490855601CC4B2642CEF
:10181000F8DB002096490870FFF7EAFF10BD10B50D
:1018200094A000F073FC4FF4967000F0B8FA93A106
:101830008E4800F0D4FC92490860FFF7DDFF0EE00F
:10184000FFF7DAFF8BA000F061FC4FF4967000F018
:10185000A6FA8AA1854800F0C2FC89490860884838
:1018600000680028ECD087A000F050FC4FF4967080
:1018700000F095FA86A000F049FC4FF4967000F055
:101880008EFA87A000F042FC4FF4967000F087FAC1
:1018900086A1764800F0A3FC79490860FFF7ACFF09
:1018A0000EE0FFF7A9FF7EA000F030FC4FF4967029
:1018B00000F075FA7DA16D4800F091FC7049086058
:1018C0006F4800680028ECD079A000F01FFC4FF4AE
:1018D000967000F064FA69A1644800F080FC6849E1
:1018E0000860FFF789FF76A000F010FC4FF49670B7
:1018F00000F055FA75A15D4800F071FC6049086080
:10190000FFF77AFF0EE0FFF777FF6DA000F0FEFB18
:101910004FF4967000F043FA6CA1544800F05FFC5D
:1019200057490860564800680028ECD06AA000F0CB
:10193000EDFB4FF4967000F032FA6AA14B4800F0CC
:101940004EFC4F4908600846006810B3084600681E
:10195000007A30380968C979303901EB810100EB30
:1019600041006249087008460078632804D0444862
:101970000068C079303840B906E000205B4981F842
:1019800072005BA000F06AFBF7E70120574981F87D
:101990007200FFF731FF10BD10B55CA000F0B6FB80
:1019A0004FF4967000F0FBF965A1304800F017FC89
:1019B0003349086008E062A12C4800F010FC30496F
:1019C0000860642000F0EBF92D4800680028F2D090
:1019D000FFF712FF10BD70B504460D462A4621469A
:1019E0005BA000F093FB4FF4967000F0D8F908E08C
:1019F0005CA11E4800F0F3FB21490860642000F060
:101A0000CEF91F4800680028F2D0184800F015FBF6
:101A100000201749087070BD70B504460D462A466F
:101A2000214652A000F072FB4FF4967000F0B7F917
:101A300008E04CA10D4800F0D2FB11490860642079
:101A400000F0ADF90E4800680028F2D0FFF7D4FE90
:101A500070BD10B54BA1054800F0C1FB08490860F6
:101A60000846006808B1FFF7C7FE10BDB7000020A8
:101A70004000002041540D0A000000004F4B0000C0
:101A80002800002041542B4346554E3D310D0A009D
:101A900041542B5149434C4F53453D300D0A0000F2
:101AA00041542B43494D490D0A00000034363000A3
:101AB00041542B43474154543D310D0A000000006E
:101AC00041542B43474154543F0D0A002B43474197
:101AD00054543A203100000041542B434553510DDA
:101AE0000A0000002B434553510000004400002031
:101AF000D0C5BAC5CBD1CBF7CAA7B0DCA3ACC7EB76
:101B0000B2E9BFB4D4ADD2F2210D0A0041542B5139
:101B1000494F50454E3D312C302C22544350222CFD
:101B20002234372E39322E3134362E323130222CB7
:101B3000383838382C313233342C310D0A0000005B
:101B40002B51494F50454E3A20302C3000000000B8
:101B500041542B514953454E443D302C25732C257F
:101B6000730D0A0053454E44204F4B0041542B51F6
:101B70004953454E4445583D302C25732C25730D53
:101B80000A0000002B2B51495552433A0000000037
:101B900010B56048006820F0F0005E490860084613
:101BA000006840F03000086000205B4908601420A5
:101BB00000F0F5F801205949C1F884011E2000F019
:101BC000CAF810BD10B500245248006820F0F0009B
:101BD000504908600846006840F08000086004E052
:101BE000601CC4B2012000F0B6F84B488038006891
:101BF00008B1642CF4DB642C01DB012010BD00244F
:101C000004E0601CC4B2012000F0A5F8424880380E
:101C1000006808B9642CF4DB642C01DB0120EDE7DB
:101C20000020EBE710B5002404E0601CC4B20120E2
:101C300000F091F838488038006808B1642CF4DB73
:101C4000002404E0601CC4B2012000F084F8324893
:101C50008038006808B9642CF4DB282000F07BF899
:101C60002D488038006808B1012010BD0020FCE735
:101C700070B50024002506E06006040EFFF7D2FFD1
:101C80000443681CC5B2082DF6DB204670BD7CB548
:101C900005460E46FFF77CFFFFF794FFF8B90024D6
:101CA00005E0FFF7E5FF0DF80400601CC4B2052C49
:101CB000F7DB9DF800009DF8011008449DF8021024
:101CC00008449DF8031008449DF80410884208D188
:101CD0009DF8000030709DF80200287001E001209E
:101CE0007CBD0020FCE710B50D48806940F008007D
:101CF0000B4988610748006820F07040054908607A
:101D00000846006840F030000860FFF741FFFFF729
:101D100059FF10BD000C0140848121420080214206
:101D20000010024010B56FF00400FEF76AFC2E4868
:101D300000682E49B0FBF1F02D4908700846007884
:101D400000EB4001C1EBC0104FF6FF7101EAC0008B
:101D50002849088010BD0146254A12784A434FF0B1
:101D6000E0235A6100229A611A46126942F0010288
:101D70001A6100BF4FF0E022106900F001021AB1B1
:101D800000F48032002AF5D04FF0E022126922F0F0
:101D900001024FF0E0231A6100229A617047014668
:101DA000144A12884A434FF0E0235A6100229A6194
:101DB0001A46126942F001021A6100BF4FF0E02298
:101DC000106900F001021AB100F48032002AF5D047
:101DD0004FF0E022126922F001024FF0E0231A6175
:101DE00000229A61704700000000002000127A0073
:101DF000320000203400002010B54FF4A060FEF740
:101E0000B1FB10BD00BF704700BFB84A128802F096
:101E10004002002AF9D0C2B2B44B1B1D1A80704791
:101E200010B5044600BF8021B148FFF731FC0028FF
:101E3000F9D02146AE48FFF7BDFB10BD10B50446F2
:101E400000BF8021A948FFF723FC0028F9D02146D4
:101E5000A648FFF7AFFB10BD10B586B004460121C0
:101E600044F20400FFF706FAA148FFF767FA4FF4BF
:101E70000070ADF8140003208DF8160018208DF8BE
:101E8000170005A99B48FEF719FF4FF48060ADF8D5
:101E9000140048208DF8170005A99648FEF70EFF9C
:101EA00025208DF8000003208DF801008DF8020038
:101EB00001208DF803006846FEF759FB01940020CD
:101EC000ADF80800ADF80A00ADF80C00ADF8100050
:101ED0000C20ADF80E0001A98548FFF772FA012227
:101EE00040F225518248FFF704FB01218048FFF7AB
:101EF000F4FA06B010BD10B586B0044601210420E6
:101F0000FFF7B8F901214804FFF7C1F97748FFF757
:101F100015FA0420ADF8140003208DF816001820DF
:101F20008DF8170005A97348FEF7C8FE0820ADF824
:101F3000140004208DF8170005A96E48FEF7BEFEB8
:101F400026208DF8000000208DF8010001208DF87A
:101F500002008DF803006846FEF709FB019400209B
:101F6000ADF80800ADF80A00ADF80C00ADF81000AF
:101F70000C20ADF80E0001A95C48FFF722FA0122FF
:101F800040F225515948FFF7B4FA01215748FFF7AD
:101F9000A4FA06B010BD10B586B004460121082091
:101FA000FFF768F901218804FFF771F95248FFF73C
:101FB000C5F94FF48060ADF8140003208DF81600C9
:101FC00018208DF8170005A94C48FEF777FE4FF44E
:101FD0000060ADF8140004208DF8170005A94748EB
:101FE000FEF76CFE27208DF8000000208DF8010020
:101FF00001208DF802008DF803006846FEF7B7FA5D
:1020000001940020ADF80800ADF80A00ADF80C000E
:10201000ADF810000C20ADF80E0001A93648FFF70E
:10202000D0F9012240F225513348FFF762FA01212D
:102030003148FFF752FA06B010BD0BE000BF2C4943
:10204000098801F040010029F9D00178284A121DC1
:102050001180401C01780029F0D170470BE000BFCF
:102060002549098801F040010029F9D00178224A68
:10207000121D1180401C01780029F0D1704710B565
:1020800040F225511A48FFF719FB18B11848FFF71D
:1020900095FAC4B210BD10B540F225511348FFF7B0
:1020A0000DFBB0B11148FFF789FAC4B20F48FFF732
:1020B00085FAC1B2124802780078401C104B1870A3
:1020C0001048815418460078632802DD0020194624
:1020D000087010BD10B540F225510748FFF7EEFA21
:1020E00018B10548FFF76AFAC4B210BD00440040B9
:1020F000003801400008014000480040000C014049
:1021000040000020B7000020704700000FB40449D1
:1021100010B503AA029800F08FF810BC5DF814FB0C
:102120003C0000202DE9F0410E46044600202062CC
:102130002046E168884730B3252805D0D4E901213D
:102140009047206A401CF2E7E16820460027884754
:10215000050018D0A5F14100192802D820354FF408
:1021600000673246294620462760FDF7F9FF40B157
:10217000012804D0F61D26F007060836D8E7361DDC
:10218000D6E72846DAE7206ABDE8F08170B50C464C
:102190000546012A05D02878800600D5EA69002383
:1021A00002E0012305E05B1C934202D2E05C0028C0
:1021B000F9D1A869E618C01AA861286A18442862EB
:1021C0002846AFF3008004E0D5E9012114F8010BA3
:1021D0009047B442F8D32846AFF3008070BD30B5C5
:1021E00005460B462A4613F8014B12F8010B08B1BD
:1021F000A042F8D01CB1002802D06D1CF1E728469F
:1022000030BD704770477047704710B5436913B1D0
:10221000AFF3008001E0FFF7B9FF012010BD127895
:1022200000F124010A7000224A700122EDE71168D2
:102230004FF0FF32E9E70000074B70B50D467B44D5
:1022400000F011F80446284600F020F810B14FF0D5
:10225000FF3070BD204670BDC7FBFFFF01694A1CFF
:1022600002610878704700B58FB0CDE901310021D7
:10227000059105497944CDE9031011466846FFF7F9
:1022800051FF0FB000BD0000E5FFFFFF007B00F035
:1022900080007047754600F029F8AE460500694693
:1022A000534620F00700854618B020B5FFF758FACE
:1022B000BDE820404FF000064FF000074FF0000847
:1022C0004FF0000B21F00701AC46ACE8C009ACE8C8
:1022D000C009ACE8C009ACE8C0098D4670470446A7
:1022E000AFF300802046FDF74DFF00000048704727
:1022F000800100201423000800000020440000009A
:102300002801000858230008440000209C07000012
:102310004401000800A24A04000000000000000080
:10232000010203040607080900000000010203047B
:102330000102030406070809020406080000000061
:10234000000000000000000000000000000000008D
:08235000000000000000000085
:04000005080000ED02
:00000001FF
